:100000000C942A001895000018950000189500001F
:10001000189500001895000018950000189500002C
:10002000189500001895000018950000189500001C
:10003000189500001895000018950000189500000C
:1000400018950000189500001895000018950000FC
:10005000189500008FE58DBFC0E4E6E24E2E88E0E3
:100060008EBFD8E0F8E05F2EEEEFF7E0A0E6B0E05C
:1000700088278D933197E9F787E689B980E080BDBD
:1000800088E18AB984B7082E877F84BF8FE181BD5C
:1000900087E081BD0E944902662487E886B980EC2A
:1000A00087B98CE00E9497020E942E028FE713E02E
:1000B0000E943D02E4EAF9E00E9427028FEB15E07E
:1000C0000E943D02E0EBF9E00E942702E2E0F0E04E
:1000D0000E9440020E942E02379A07B1007E006003
:1000E00007B90E94C203A0E6B0E08D939C9307B1CC
:1000F000007E016007B90E94C203A2E6B0E08D93C2
:100100009C93E0EAF9E00E946104E0E6F0E0D1901F
:10011000E080FF2400270E94EF030E942D04EDE001
:10012000F0E0A4E6B0E00E94C404E0EAF9E00E9436
:100130006104E2E6F0E0D190E080FF2400270E9415
:10014000EF030E942D04EDE0F0E0A3E7B0E00E9491
:10015000C404E3E7F0E00E94D003E4E6F0E00E948C
:10016000CB030E942D04EDE0F0E0A2E8B0E00E9495
:10017000C404AEE0B8E0AF93BF93E4E6F0E00E94C1
:10018000CB030E94D90211E002E0BF91AF910E941F
:100190007704EEE0F8E0A8E6B0E00E94BF04A8E62D
:1001A000B0E00E94CA04082F043011F00C94FE0045
:1001B0008CE00E94D302E8E6F0E0A881B9810E94B9
:1001C000BF04A8E6B0E0E8EBF9E00E94BC03E881D8
:1001D000F981A8E6B0E00E9418020E94BF04A8E6D8
:1001E000B0E00E941802EAEBF9E00E94BC038CE048
:1001F000481A8827580A22960C940601A8E6B0E00F
:100200000E941802EAEBF9E00E94BC038FE711E0BC
:100210000E943D02A8E6B0E00E942102AEE0B8E0F4
:10022000AF93BF93E3E7F0E00E94CB030E94D902B3
:1002300011E002E0BF91AF910E947704EEE0F8E098
:10024000A7E7B0E00E94BF04A7E7B0E00E94CA049D
:10025000082F043011F00C9453018CE00E94D3025B
:10026000E7E7F0E0A881B9810E94BF04A7E7B0E00A
:10027000E8EBF9E00E94BC03E881F981A7E7B0E070
:100280000E9418020E94BF04A7E7B0E00E94180273
:10029000ECEBF9E00E94BC038CE0481A8827580A6E
:1002A00022960C945B01A7E7B0E00E941802ECEBE9
:1002B000F9E00E94BC038FEB11E00E943D02A7E72A
:1002C000B0E00E942102AEE0B8E0AF93BF93E2E855
:1002D000F0E00E94CB030E94D90211E002E0BF913E
:1002E000AF910E947704EEE0F8E0A6E8B0E00E944B
:1002F000BF04A6E8B0E00E94CA04082F043011F041
:100300000C94A6018CE00E94D302E6E8F0E0A881FC
:10031000B9810E94BF04A6E8B0E0EEEBF9E00E94CC
:10032000BC03E881F981A6E8B0E00E9418020E94AF
:10033000BF04A6E8B0E00E941802E2ECF9E00E94D7
:10034000BC038CE0481A8827580A2296A6E8B0E039
:100350000E94CA04082F053011F00C94D3018CE0E0
:100360000E94D302E6E8F0E0A881B9810E94BF04B0
:10037000A6E8B0E0E4ECF9E00E94BC03E881F98172
:10038000A6E8B0E00E9418020E94BF04A6E8B0E010
:100390000E941802E2ECF9E00E94BC038CE0481ACB
:1003A0008827580A2296A6E8B0E00E94CA04082FBF
:1003B000063011F00C9400028CE00E94D302E6E8B3
:1003C000F0E0A881B9810E94BF04A6E8B0E0E8EBA4
:1003D000F9E00E94BC03E881F981A6E8B0E00E9440
:1003E00018020E94BF04A6E8B0E00E941802E2ECE6
:1003F000F9E00E94BC038CE0481A8827580A22962C
:100400008FE718E00E943D02A6E8B0E00E942102BA
:100410008FEB19E00E943D02E8ECF9E00E94270210
:100420008AEF90E00E94C4020C946D00F894FFCF14
:100430008F938D918823E9F711978F910895AEE0FE
:10044000B8E08D91882311F06CD0FBCF08950E9405
:100450005D04802D11F065D0FACF089581E067D05A
:1004600015D080E864C08FE7213039F08FEB22305F
:1004700021F08FE8233009F08FEC810F0C94970264
:1004800088EE93E081D03197D9F7089583E09927DA
:100490007BC08AEF90E00E94C402BF9ABE9ABD9AC8
:1004A000BC9ABB9ABA9AC29885E090E00E94C402B6
:1004B000C398C798C698C59AC49AC39AEF93FF93F6
:1004C000ECE8F1E00E94B802FF91EF91C39859D097
:1004D000C39AEF93FF93ECE8F1E00E94B802FF911A
:1004E000EF91C3984ED0C39AEF93FF93ECE8F1E0FD
:1004F0000E94B802FF91EF91C39843D0C498C39A69
:10050000EF93FF93ECE8F1E00E94B802FF91EF91C6
:10051000C39837D088E20BD08EE009D086E007D0B0
:100520000895C29A829505D004D02BD00895C29820
:10053000F9CF859510F4C49A01C0C498859510F43C
:10054000C59A01C0C598859510F4C69A01C0C69891
:10055000859510F4C79A01C0C798C39AEF93FF938B
:10056000ECE8F1E00E94B802FF91EF91C398089582
:100570003197F1F70895689462F80895E89462F865
:10058000089581E090E000C0EF93FF93EE27E82B01
:10059000E92B31F0E0EAFFE03197F1F70197D1F76D
:1005A000FF91EF9108955A924A92480E8827581E5B
:1005B00008958DE207FD8D938F2D881F802F881F52
:1005C0008F57082F6894F7F8802F87FF15C0809504
:1005D0008395082F80E38D938EE28D93802F815237
:1005E00028F080E38D9399279C93089544270A95DA
:1005F000802F09F196D01FC0805230F09EE49D9369
:1006000081E48D939D93EFCF4427DF92EF92FF9289
:100610000F938FE1801B11F0082F83D089D09EE2C9
:100620009D930F91FF90EF90DF9044270395003248
:1006300009F4D7CF2BD03F93E2ECF6E038E12F2D31
:100640001E2D0D2DFF24EE24DD244427000F111F45
:10065000221FA8F42F923F920E945D04102C0E944A
:100660005D04202C0E945D04302C0E945D043197B3
:10067000410DD21CE31CF01C3F902F9001C033961B
:1006800031963A9519F73F9107D0AFCFDD0CEE1CAC
:10069000FF1C0A95D9F70895002719E058D08F93C9
:1006A000802B11F0039501C08F911A95B9F7802F17
:1006B000882309F496CF8F91805D8D930A95D9F7A1
:1006C00092CF0065CD1D80B2E60E40597307A0ACF5
:1006D000B90350D6DC01286BEE0094357700CA9A36
:1006E0003B0065CD1D00B2E60E0059730700ACB9A2
:1006F0000300D6DC01006BEE0000357700009A3B6A
:100700000000CD1D0000E60E000073070000B903D5
:100710000000DC010000EE000000770000003B005C
:100720000000F694E794D79447950A95D1F7089579
:1007300000270DD08F9303958F2D8E298D29842B23
:10074000C1F78F91805D8D930A95D9F74CCF1F9398
:100750000F93002710E2440FDD1CEE1CFF1C001F4E
:10076000802F9AE0890B10F0082F43951A9599F77E
:10077000802F0F911F9108950E945D040D9200201B
:10078000D9F70895369A3699FECF369A3699FECF24
:1007900084B195B10895D190E190F19001910895BF
:1007A00021913191419151910895102F90E8FF0CC2
:1007B000001F0927990FF7941078652F90E8440FD0
:1007C000551F5927990F4795607800380895FF0CF9
:1007D00090E89027110F9795F794092F0895102FFF
:1007E000BD2CDE2CEF2CF02E11234AF4B094D094C3
:1007F000E094F0949FEFB91AD90AE90AF90A0EE1D8
:10080000FF2039F4FE2CED2CDB2CBB240850C2F762
:100810001EC032F00A95BB0CDD1CEE1CFF1CF9CF8C
:1008200001D0D5CFB7FE089590E8B91611F4D0FEE7
:1008300008959FEFD91AE90AF90A09F40395089572
:100840009FE7092FF92A9FEFD92EE92E0895DD247D
:10085000EE24FF24002711270895A7DFC1F35038A5
:10086000B1F31627005850580894051F12F418F4D5
:10087000E7CF08F0ECCF0AD0FF202AF0BB0CDD1C3C
:10088000EE1CFF1CA4CF0F5FDBF2A1CF9F92992437
:10089000AA24BB24992788E1990CAA1CBB1CDD1C47
:1008A000EE1CFF1C30F4920EA31EB41ED91EE91ECE
:1008B000F91E8A9589F79F900895C8953196002072
:1008C0000895FBDF202DF9DF302DF7DF402DF5DF18
:1008D000502D089599278D9193958823E1F793954D
:1008E00011968C9311978E919A95D1F70895EA2FCE
:1008F000FB2F00244C918D9103948E32E1F711244B
:100900008D9113948823E1F71A94101640F41197EF
:10091000202F2119239580E38D932A95E9F7113033
:1009200039F59927AE2FBF2FA00DB91FA00FB91F02
:100930008C919C93853308F421C031E08E918E32E6
:10094000E9F38D3241F0830F8A3319F480E331E00B
:1009500001C033278C93AE1789F7332341F0AE2FB4
:10096000BF2FB8DF81E34D3209F4319680830895BB
:100970008827E00DF81FE00FF81F8083089581910C
:100980008D938823E1F7089594E081918D939A9552
:10099000E1F708958FEF83959D919923E1F70895ED
:1009A0000000483D20576174746D657465720000E5
:1009B000444C334A494E000020005600410020209C
:1009C00020005700202000007878782E7979576829
:0209D000000025
:00000001FF
